:1000000000308A00412900000A108A100A11820774
:1000100028340C34013406340A108A100A1182077D
:100020004234613474346534723469346534203454
:100030006A34653420346E34613462346934743423
:10004000613420346E34613400340A108A100A118D
:100050008207613420346E346134703461346A3420
:1000600065346E34693420347A3461346A346934E6
:100070007334743475346A34653400340A108A1069
:100080000A118207413454342B344334423443340C
:100090000D3400340A108A100A11820725346334A3
:1000A000253463342034703472346F3463346534EF
:1000B0006E34743400340A108A100A1182076234D4
:1000C00061347434653472346934653400343730E3
:1000D00084008313000803197E280130F800BF3024
:1000E000F7006400F70B7128F80B6F284A30F7000F
:1000F000F70B782800006400800B6D280034070897
:10010000F039BE003D080F393E04870006148316FF
:10011000061064002030F700F70B8C288F2883121C
:1001200006108316061083120034BB08031D9A289C
:1001300086109B288614831686108312BC0E3C08FA
:10014000BD007F20BC0E3C08BD007F206400423013
:10015000F700F70BA92800341430B7006720F030FF
:100160008316870583128610831686108312061065
:10017000831606108312B5013508023C031CC828FB
:100180000230B70067200330BD007F20B50ABC28CD
:1001900064000C30F700F70BCB28CE280230BD00EE
:1001A0007F2064000C30F700F70BD428D728B50166
:1001B0003508023C031CE82835080420B600BB01C2
:1001C0003608BC0095200230B7006720B50AD82851
:1001D000922901303802FC3E0318FB28043E062910
:1001E000B901FB284030B900FB281430B900FB28C6
:1001F0005430B900FB2801303702B907390880387C
:10020000BA00BB013A08BC00952000340A148A10D9
:100210000A118207F028F228F528F82836080C3A47
:1002200003191C29063A03192429073A03192A2914
:10023000053A03192F293429BB010130BC00952050
:100240000230B700672040290130B7000230B80003
:10025000E92040290130B700B800E9204029BB015E
:100260001030BC009520402936081F3C031C3A2959
:100270000730B6050130BB003608BC009520402988
:100280000034840183131F3083050C3083169900DA
:10029000A630980090308312980083161F149F1484
:1002A0001F159F1107309C00FF308312B400831686
:1002B0001F149F141F159F1183121F1083160912FC
:1002C00083129412B41234088316870083123416F2
:1002D0003408831687008312B4113408831687000C
:1002E0000130831294000030831694000108C7394E
:1002F00008388100831290010030F800920000302D
:100300008316920007309C00050864000230F70055
:10031000F70B88298B291C0883120D1383169D0166
:100320008312AC289630B7006720B50135080C2041
:10033000B50AF700B6000E2114303502031D9629C8
:100340000130B7000330B800E920B5013508252099
:10035000B50AF700B6000E2114303502031DA62998
:10036000B50135083E20B50AF70077080C1EB629FE
:10037000990007303502031DB12920308400831312
:100380008403840A8C1EC2291A0880000D300002E2
:10039000031DC12980018C1ECB291A08203084003E
:1003A00083138403840A8C1ED3291A0880000D301D
:1003B0000002031DD22980010630B7000230B800C8
:1003C000E9202908B6000E212A08B6000E210430C3
:1003D000B50035084A20B50AF700B6000E210C30EA
:1003E0003502031DE9292708303C031D082A073080
:1003F000B7000430B800E920B50135085B20B50A24
:10040000F700B6000E2107303502031DFD29162A1C
:100410000930B7000430B800E9207330B6000E216F
:100420006930B6000E217430B6000E210A30B500D6
:0E043000FA30B7006720B50B182AB029630018
:02400E00393F38
:00000001FF
